:020000040000FA
:200000000000000000000000000000000000000000000000000000000000000000000000E0
:200020000000000000000000000000000000000000000000000000000000000000000000C0
:200040000000000000000000000000000000000000000000000000000000000000000000A0
:20006000000000000000000000000000000000000000000000000000000000000000000080
:20090000040206010503070004020601050307000402060105030700040206010503070067
:20092000040206010503070004020601050307000402060105030700040206010503070047
:20094000040206010503070004020601050307000402060105030700040206010503070027
:20096000040206010503070004020601050307000402060105030700040206010503070007
:200980000404040404040404040404040404040404040404040404040404040404040404D7
:2009A0000404040404040404040404040404040404040404040404040404040404040404B7
:2009C000040404040404040404040404040404040404040404040404040404040404040497
:2009E000040404040404040404040404040404040404040404040404040404040404040477
:200A00000000000000000000000000000000000000000000000000000000000000000000D6
:200A20000000000000000000000000000000000000000000000000000000000000000000B6
:200A4000000000000000000000000000000000000000000000000000000000000000000096
:200A6000000000000000000000000000000000000000000000000000000000000000000076
:200A800004040404040404040909090909090909090909090909090909090909090909095E
:200AA000090909090909090909090909090909090909090909090909090909090909090916
:200AC00004040404040404040909090909090909090909090909090909090909090909091E
:200AE0000909090909090909090909090909090909090909090909090909090909090909D6
:200B0000070707070707070707070707070707070000000000000000000000000000000065
:200B200003050106020400070305010602040007000000000000000000000000000000007D
:200B4000070707070707070707070707070707070000000000000000000000000000000025
:200B600003050106020400070305010602040007000000000000000000000000000000003D
:200B8000040404040404040404040404040404040909090909090909090909090909090985
:200BA000484848484848484848484848484848480606060606060606060606060606060655
:200BC000040404040404040404040404040404040909090909090909090909090909090945
:200BE000484848484848484848484848484848480606060606060606060606060606060615
:200C0000000000000000000000000000000000000102020404080801010202040408080198
:200C2000020101080804040202010108080404020000000000000000000000000000000078
:200C4000000000000000000000000000000000000102020404080801010202040408080158
:200C6000010202040408080101020204040808010000000000000000000000000000000038
:200C8000888888888888888888888888888888888888888888888888888888888888888854
:200CA000888888888888888888888888888888888888888888888888888888888888888834
:200CC000888888888888888888888888888888888888888888888888888888888888888814
:200CE0008888888888888888888888888888888888888888888888888888888888888888F4
:200D0000000000000000000000000000000000001020204040808010102020404080801013
:200D2000010202040408080101020204040808010202020808080802020202080808080227
:200D40000000000000000000000000000000000010202040408080101020204040808010D3
:200D600001020204040808010102020404080801010101040404040101010104040404010F
:200D8000888888888888888888888888888888888888888888888888888888888888888853
:200DA000888888888888888888888888888888888888888888888888888888888888888833
:200DC000888888888888888888888888888888888888888888888888888888888888888813
:200DE0008888888888888888888888888888888888888888888888888888888888888888F3
:200E000000000000000000000000000000000000030501060204000603050106020400069C
:200E200003050106020400060305010602040006070707070707070707070707070707070C
:200E400000000000000000000000000000000000030501060204000603050106020400065C
:200E60000305010602040006030501060204000607070707070707070707070707070707CC
:200E80000404040404040404090909090909090920202020202020202020202020202020EA
:200EA000101010101010101010101010101010101010101010101010101010101010101032
:200EC0000404040404040404090909090909090920202020202020202020202020202020AA
:200EE0001010101010101010101010101010101010101010101010101010101010101010F2
:200F0000030501060204000F030501060204000F030501060204000F030501060204000F41
:200F2000030501060204000F030501060204000F030501060204000F030501060204000F21
:200F4000030501060204000F030501060204000F030501060204000F030501060204000F01
:200F6000030501060204000F030501060204000F030501060204000F030501060204000FE1
:200F8000101010101010101010101010101010101010101010101010101010101010101051
:200FA000101010101010101010101010101010101010101010101010101010101010101031
:200FC000101010101010101010101010101010101010101010101010101010101010101011
:200FE0001010101010101010101010101010101010101010101010101010101010101010F1
:201000000B0D090E0A0C000F0B0D090E0A0C000F0B0D090E0A0C000F0B0D090E0A0C000F80
:201020000B0D090E0A0C000F0B0D090E0A0C000F0B0D090E0A0C000F0B0D090E0A0C000F60
:201040000B0D090E0A0C000F0B0D090E0A0C000F0B0D090E0A0C000F0B0D090E0A0C000F40
:201060000B0D090E0A0C000F0B0D090E0A0C000F0B0D090E0A0C000F0B0D090E0A0C000F20
:20108000101010101010101010101010101010101010101010101010101010101010101050
:2010A000101010101010101010101010101010101010101010101010101010101010101030
:2010C000101010101010101010101010101010101010101010101010101010101010101010
:2010E0001010101010101010101010101010101010101010101010101010101010101010F0
:20110000030501060204000F030501060204000F030501060204000F030501060204000F3F
:201120000000000000000000000000000000000000000000000000000000000000000000AF
:20114000030501060204000F030501060204000F030501060204000F030501060204000FFF
:2011600000000000000000000000000000000000000000000000000000000000000000006F
:2011800010101010101010101010101010101010101010101010101010101010101010104F
:2011A00009090909090909090909090909090909090909090909090909090909090909090F
:2011C00010101010101010101010101010101010101010101010101010101010101010100F
:2011E0000909090909090909090909090909090909090909090909090909090909090909CF
:201200000B0D090E0A0C000F0B0D090E0A0C000F0B0D090E0A0C000F0B0D090E0A0C000F7E
:201220000000000000000000000000000000000000000000000000000000000000000000AE
:201240000B0D090E0A0C000F0B0D090E0A0C000F0B0D090E0A0C000F0B0D090E0A0C000F3E
:2012600000000000000000000000000000000000000000000000000000000000000000006E
:2012800010101010101010101010101010101010101010101010101010101010101010104E
:2012A00009090909090909090909090909090909090909090909090909090909090909090E
:2012C00010101010101010101010101010101010101010101010101010101010101010100E
:2012E0000909090909090909090909090909090909090909090909090909090909090909CE
:2013000004020601050307000402060105030700040206010503070004020601050307005D
:20132000030501060204000F030501060204000F030501060204000F030501060204000F1D
:2013400004020601050307000402060105030700040206010503070004020601050307001D
:20136000030501060204000F030501060204000F030501060204000F030501060204000FDD
:201380000404040404040404040404040404040404040404040404040404040404040404CD
:2013A00010101010101010101010101010101010101010101010101010101010101010102D
:2013C00004040404040404040404040404040404040404040404040404040404040404048D
:2013E0001010101010101010101010101010101010101010101010101010101010101010ED
:2014000004020601050307000402060105030700040206010503070004020601050307005C
:201420000B0D090E0A0C000F0B0D090E0A0C000F0B0D090E0A0C000F0B0D090E0A0C000F5C
:2014400004020601050307000402060105030700040206010503070004020601050307001C
:201460000B0D090E0A0C000F0B0D090E0A0C000F0B0D090E0A0C000F0B0D090E0A0C000F1C
:201480000404040404040404040404040404040404040404040404040404040404040404CC
:2014A00010101010101010101010101010101010101010101010101010101010101010102C
:2014C00004040404040404040404040404040404040404040404040404040404040404048C
:2014E0001010101010101010101010101010101010101010101010101010101010101010EC
:2015000003050106020400070305010602040007030501060204000703050106020400075B
:201520000305010602040007070707070707070707070707070707070707070707070707E7
:2015400003050106020400070305010602040007030501060204000703050106020400071B
:201560000305010602040007070707070707070707070707070707070707070707070707A7
:2015800010101010101010101010101010101010101010101010101010101010101010104B
:2015A00010101010101010101010101010101010101010101010101010101010101010102B
:2015C00010101010101010101010101010101010101010101010101010101010101010100B
:2015E0001010101010101010101010101010101010101010101010101010101010101010EB
:2016000004020601050307000402060105030700040206010503070004020601050307005A
:201620000402060105030700070707070707070707070707070707070707070707070707E6
:2016400004020601050307000402060105030700040206010503070004020601050307001A
:201660000402060105030700070707070707070707070707070707070707070707070707A6
:201680000404040404040404040404040404040404040404040404040404040404040404CA
:2016A0000404040404040404040404040404040404040404040404040404040404040404AA
:2016C00004040404040404040404040404040404040404040404040404040404040404048A
:2016E00004040404040404040404040404040404040404040404040404040404040404046A
:201700000000000000000000000000000000000000000000000000000000000000000000C9
:20172000000000000000000007070707070707070707070707070707070707070707070701
:20174000000000000000000000000000000000000000000000000000000000000000000089
:201760000000000000000000070707070707070707070707070707070707070707070707C1
:20178000090909090909090909090909090909090909090909090909090909090909090929
:2017A000090909090909090904040404040404040404040404040404040404040404040481
:2017C0000909090909090909090909090909090909090909090909090909090909090909E9
:2017E000090909090909090904040404040404040404040404040404040404040404040441
:20180000040206010503070004020601050307000402060105030700040206010503070058
:201820000000000000000000000000000000000000000000000000000000000000000000A8
:20184000040206010503070004020601050307000402060105030700040206010503070018
:20186000000000000000000000000000000000000000000000000000000000000000000068
:201880000404040404040404040404040404040404040404040404040404040404040404C8
:2018A000090909090909090909090909090909090909090909090909090909090909090908
:2018C000040404040404040404040404040404040404040404040404040404040404040488
:2018E0000909090909090909090909090909090909090909090909090909090909090909C8
:20190000040206010503070004020601050307000402060105030700030501060204000F4F
:20192000030501060204000F00000000000000000000000000000000000000000000000083
:20194000040206010503070004020601050307000402060105030700030501060204000F0F
:20196000030501060204000F00000000000000000000000000000000000000000000000043
:20198000040404040404040404040404040404040404040404040404101010101010101067
:2019A0001010101010101010090909090909090909090909090909090909090909090909CF
:2019C000040404040404040404040404040404040404040404040404101010101010101027
:2019E00010101010101010100909090909090909090909090909090909090909090909098F
:201A000004020601050307000402060105030700030501060204000F00000000000000006A
:201A200003050106020400070305010602040007000000000000000000000000000000006E
:201A400004020601050307000402060105030700030501060204000F00000000000000002A
:201A600003050106020400070305010602040007000000000000000000000000000000002E
:201A800004040404040404040404040404040404101010101010101009090909090909093E
:201AA000484848484848484848484848484848480606060606060606060606060606060646
:201AC0000404040404040404040404040404040410101010101010100909090909090909FE
:201AE000484848484848484848484848484848480606060606060606060606060606060606
:201B000004020601050307000402060105030700030501060204000F000000000000000069
:201B2000102020404080801001020204040808010202020808080802020202080808080257
:201B400004020601050307000402060105030700030501060204000F000000000000000029
:201B600010202040408080100102020404080801010101040404040101010104040404013F
:201B800004040404040404040404040404040404101010101010101009090909090909093D
:201BA000888888888888888888888888888888888888888888888888888888888888888825
:201BC0000404040404040404040404040404040410101010101010100909090909090909FD
:201BE0008888888888888888888888888888888888888888888888888888888888888888E5
:201C000004020601050307000402060105030700030501060204000F000000000000000068
:201C20000305010602040006030501060204000607070707070707070707070707070707FE
:201C400004020601050307000402060105030700030501060204000F000000000000000028
:201C60000305010602040006030501060204000607070707070707070707070707070707BE
:201C800004040404040404040404040404040404101010101010101009090909090909093C
:201CA0002020202020202020101010101010101010101010101010101010101010101010A4
:201CC0000404040404040404040404040404040410101010101010100909090909090909FC
:201CE000202020202020202010101010101010101010101010101010101010101010101064
:201D0000030501060204000703050106020400070501060204000703010602040007030553
:201D2000060204000703050102040007030501060400070305010602040007030501060233
:201D4000030501060204000703050106020400070501060204000703010602040007030513
:201D60000602040007030501020400070305010604000703050106020400070305010602F3
:201D8000101010101010101010101010101010101010101010101010101010101010101043
:201DA000101010101010101010101010101010101010101010101010101010101010101023
:201DC000101010101010101010101010101010101010101010101010101010101010101003
:201DE0001010101010101010101010101010101010101010101010101010101010101010E3
:201E0000030303030303030303030303030303030505050505050505010101010101010162
:201E2000060606060606060602020202020202020404040404040404040404040404040422
:201E4000030303030303030303030303030303030505050505050505010101010101010122
:201E60000606060606060606020202020202020204040404040404040404040404040404E2
:201E8000101010101010101010101010101010101010101010101010101010101010101042
:201EA000101010101010101010101010101010101010101010101010101010101010101022
:201EC000101010101010101010101010101010101010101010101010101010101010101002
:201EE0001010101010101010101010101010101010101010101010101010101010101010E2
:201F0000070707070707000007070707070700000700000000070000070007070007000043
:201F2000070007070007000007000000000700000707070707070000070707070707000023
:201F4000070707070707000007070707070700000700000000070000070007070007000003
:201F60000700070700070000070000000007000007070707070700000707070707070000E3
:201F80000404040404040404040404040404040404040404040404040404040404040404C1
:201FA0000404040404040404040404040404040404040404040404040404040404040404A1
:201FC000040404040404040404040404040404040404040404040404040404040404040481
:201FE000040404040404040404040404040404040404040404040404040404040404040461
:00000001FF
